:100000000C94E9000C9440070C9490070C940601A2
:100010000C9406010C9406010C9406010C94060144
:100020000C9406010C9406010C9406010C941F0616
:100030000C94DA050C9406010C9406010C9406014C
:100040000C9406010C9406010C9409080C94080108
:100050000C940601165452494747455200000015BA
:1000600054494D454F5554000000145354415455C4
:1000700053000000001353504F4C4C000000000090
:100080001253454E440000000000001152455350E9
:100090004F4E534500001052455345540000000098
:1000A000000F524551554553540000000E52454D26
:1000B0004F5445000000000D50504F4C4C000000C4
:1000C00000000C504153530000000000000B4F553E
:1000D00054505554000000000A4F4E4C494E450004
:1000E000000000094F46464C494E45000000084CB0
:1000F0004F43414C0000000000074C414E47454F24
:10010000530000000647504942454F530000000588
:100110004552525452415000000004454E5445523D
:10012000000000000003434F4E464947555245002A
:1001300002434C45415200000000000141424F5231
:10014000540000000000014C4F434B4F5554000039
:1001500000014F555400000000000000024C460012
:100160000000000000000003494E000000000000F5
:10017000000004454E44000000000000000543520A
:10018000000000000000000006434852000000008C
:100190000000000741534300000000000000282534
:1001A000752900257500014E4F454E4400000000A2
:1001B0000002454E440000000000000025750025A7
:1001C00075002575006364696E6F70737578585B90
:1001D000000011241FBECFE5D4E0DEBFCDBF10E08C
:1001E000A0E6B0E0E0E5FCE102C005900D92A23887
:1001F000B107D9F711E0A2E8B0E001C01D92AF3A13
:10020000B107E1F70E9463010C94260E0C940000E4
:100210001F920F920FB60F9211242F933F938F933B
:100220009F93809182008F5F8093820081508830FD
:1002300008F440C010928200809183008F5F809309
:100240008300803190F0109283008091970190910B
:1002500098019093870080938600809195019091FA
:1002600096019093850080938400209186003091C0
:100270008700922F91709295907F88B38F7E892B03
:1002800088BB369527953093870020938600209170
:10029000840030918500922F9170990F990F990FDA
:1002A00088B3877F892B88BB369527953093850047
:1002B000209384009F918F913F912F910F900FBEBB
:1002C0000F901F9018958DE78CBF8DE083BF89B785
:1002D000826089BFC39AC49887B3886B87BBBE9876
:1002E0000E9429090E949C010E94CE060E943E099C
:1002F0000E94A50178940E94D503FDCF89E991E081
:100300006EE070E04EE050E00E94C00D08950F9343
:100310001F9309E911E0C80160E070E04EE050E091
:100320000E94B00DC8016EE070E04EE050E00E9407
:10033000C00D1F910F91089589E991E06EE070E082
:100340004EE050E00E94B00D089510928800109287
:1003500096011092950108950E94E20781E00E94A3
:10036000F3080895CF93DF938091A9019091AA019A
:100370000E946D0AEC010E94580A892BA9F760912E
:10038000A9017091AA01CE010E94010BDF91CF91CA
:100390000895AF92BF92CF92DF92EF92FF920F93A8
:1003A0001F93DF93CF9300D0CDB7DEB78FE50E94C8
:1003B000B30780E290E09A838983EE24FF2433EA36
:1003C000A32E31E0B32E6E010894C11CD11C00D0C5
:1003D00000D0EDB7FEB7B282A182D482C3820E9460
:1003E000DB0A8C010F900F900F900F9081309105D8
:1003F000B9F40E94B20189819A81809728F0109304
:100400009801009397010CC0FCE2EF16F10419F07B
:100410008FE30E94B30789818F7180620E94B307C6
:100420008091A9019091AA010E946D0A2CE2E22E0E
:10043000F12C8C32910559F26091A9017091AA01B9
:100440000E94010B20E089819A81809708F421E0C5
:10045000822F0F900F90CF91DF911F910F91FF90FE
:10046000EF90DF90CF90BF90AF900895BF92CF9262
:10047000DF92EF92FF920F931F93CF93DF937C0154
:10048000C62E0E94B2018091A9019091AA010E94FA
:100490006D0AEC0100E0DD244BE0B42E43C0DB9C90
:1004A000F0011124EE0DFF1D802F90E00196E80F62
:1004B000F91F1491CE010E94600A212F30E0281705
:1004C000390749F48091A9019091AA010E946D0A0F
:1004D000EC010F5F27C07D2D7F5F7C1540F57B9D74
:1004E000C0011124D701A80FB91FAC014B505040D7
:1004F0004E0D5F1D90E011C0292F30E02F5F3F4F60
:10050000FD01E20FF31F6491662349F0240F351FAC
:10051000F9018491681719F49F5F901768F3901799
:1005200031F4D72EFFEFCF3FDF0709F0B8CF60914E
:10053000A9017091AA01CE010E94010B002311F4C0
:1005400080E007C0EBE0DE9EF0011124EE0DFF1D00
:100550008491DF91CF911F910F91FF90EF90DF90E9
:10056000CF90BF9008952F923F924F925F926F92DB
:100570007F928F929F92AF92BF92CF92DF92EF9233
:10058000FF920F931F93DF93CF93CDB7DEB72897DA
:100590000FB6F894DEBF0FBECDBF382E292E5B01FB
:1005A0004A01DE0113969C01F90186E001900D924B
:1005B0008150E1F79D818885A114B10411F4442490
:1005C00002C0F50140808114910411F4552402C049
:1005D000F4015080D82EE92ECC24E1E06E2E712C4F
:1005E00004C0552472E0C72EDD2481E591E067E068
:1005F0000E943602F82EF4E08F17F1F0F81750F051
:1006000082E0F816B1F08F1578F091E0F91609F054
:1006100040C0E7CFE6E08E1719F18E1708F463C0EB
:10062000F7E08F17B1F545C04424CC24C394EE24E1
:100630007FC00AE010E059C08C2DC0FE0AC0A11492
:10064000B10419F04424439404C07092980160925C
:10065000970181FFCACF8114910409F08AC03EC07E
:1006600000D000D08EE991E0EDB7FEB79283818390
:1006700081E090E08C0F9D1F948383830E94DB0AAE
:100680000F900F900F900F90019741F509811A81FB
:100690002CC08091A9019091AA010E946D0A873215
:1006A000910539F06091A9017091AA010E94010B96
:1006B0003FC08091A9019091AA010E946D0A8C010E
:1006C0000E94520A892B19F067E0F62E0EC0609145
:1006D000A9017091AA01C8010E94010B70929801B2
:1006E0006092970182CF0DE010E0CC2031F44424D9
:1006F000552453E0C52EDD24EE248C2DC0FE0BC006
:1007000091E09E1540F0E3E0F0E0EC0FFD1FEE0DF0
:10071000F11D0083E39481FF0BC0E1E0ED1540F093
:10072000E6E0F0E0EC0FFD1FED0DF11D0083D3942A
:10073000FF2009F05ACFCC2011F4DD24EE240E94D2
:10074000B201ED82D886832D922D9C01D901FE0144
:10075000339686E001900D928150E1F7A114B10427
:1007600011F0F50140828114910431F0F4015082BE
:1007700003C05524539439CF28960FB6F894DEBFA2
:100780000FBECDBFCF91DF911F910F91FF90EF90E2
:10079000DF90CF90BF90AF909F908F907F906F90A1
:1007A0005F904F903F902F900895EF92FF920F939C
:1007B0001F93DF93CF9300D000D0CDB7DEB78091E9
:1007C000A9019091AA010E94680A84E590E066E17F
:1007D0000E943602182F882389F4E091A901F09134
:1007E000AA01838185FDDBC181E090E090939801AF
:1007F00080939701CF010E946D0AD1C11092980198
:1008000010929701873039F1883028F48130A1F0B7
:10081000863099F52BC08A3049F08031C9F0893093
:1008200061F50E94D30810928800AAC10E94E408D2
:1008300081E080938800A4C10E94D3080E94E4084C
:10084000109388000E94220981E00E94F30898C159
:100850000E94870108C089E991E060E070E040E013
:1008600050E00E94B3020E947E018AC18FE991E0AC
:1008700065EA71E046EA51E0F4CF80918800882370
:1008800009F487C1183021F1193030F4123061F0C9
:10089000143009F07EC1DCC01E3091F0163181F1B8
:1008A0001B3009F076C134C00E9422090E94AC01BD
:1008B0000E94C901882311F084E01AC084E125C098
:1008C00081E00E9418090E94AC010E94C90158C130
:1008D0000E94AC0186E491E061E00E943602813022
:1008E00011F481E112C00E94C901882329F081E03E
:1008F0000E94B3078FE309C080E00E94180940C13D
:100900000E94AC010E94C90188E00E94B30738C16F
:100910000E94AC010E94C90186EA91E062E00E9457
:1009200036028823A1F000E0823009F401E08091D2
:10093000A601081771F00E94FF078823E1F30093D6
:10094000A60180E0002309F481E0082F02C0009195
:10095000A6010E94B2018091A9019091AA010E9472
:100960006D0A8332910511F010E023C000D000D051
:100970008CEB91E0EDB7FEB792838183CE010196B7
:10098000948383830E94DB0A0F900F900F900F9047
:10099000019711F411E007C081E090E09093980175
:1009A0008093970110E08091A9019091AA010E9483
:1009B0006D0A8B339105D1F580E00E94F308112375
:1009C000B9F427C08091A9019091AA010E946D0AF3
:1009D000FFEF8F3F9F0739F06091A7017091A80149
:1009E0000E94AF0A08C0F0929801E092970103C0FC
:1009F000F1E0EF2EF12C89819A8101979A83898306
:100A0000019601F719C06091A7017091A8010E9499
:100A1000AF0A8091A9019091AA010E946D0A2FEF5F
:100A20008F3F920781F70E94F60906C06091A901E5
:100A30007091AA010E94010B8091A601081709F488
:100A40009FC00E94FF078823E1F30093A60198C08E
:100A500000D000D082EC91E0EDB7FEB792838183A5
:100A6000CE010396948383830E94DB0A9C010F903E
:100A70000F900F900F908130910599F48B819C819C
:100A8000809728F030939801209397010AC00E9424
:100A9000AC018FE50E94B3078B818F7180640E9447
:100AA000B3070E94B2018091A9019091AA010E940E
:100AB0006D0A83329105E9F400D000D08FEB91E00C
:100AC000EDB7FEB792838183CE0101969483838331
:100AD0000E94DB0A0F900F900F900F90019711F476
:100AE00011E00EC081E090E090939801809397010F
:100AF00006C06091A9017091AA010E94010B10E04B
:100B00008091A7019091A8010E94680A0E94910813
:100B100080E00E94F3081123B9F426C08091A70158
:100B20009091A8010E946D0AFFEF8F3F9F0739F057
:100B30006091AB017091AC010E94AF0A07C01093A5
:100B400098010093970102C001E010E089819A8129
:100B500001979A838983019609F710C06091AB01D0
:100B60007091AC010E94AF0A8091A7019091A801F9
:100B70000E946D0A2FEF8F3F920781F70E944B0A68
:100B80000E94B201E091A901F091AA01838185FD43
:100B900006C081E090E090939801809397010F90B8
:100BA0000F900F900F90CF91DF911F910F91FF90B9
:100BB000EF9008951F920F920FB60F9211248F930A
:100BC0009F93EF93FF939091CA008091C90098176B
:100BD00079F0E92FF0E0E757FF4F80818CB9892F3A
:100BE0008F5F8093CA00803420F01092CA0001C049
:100BF0005598FF91EF919F918F910F900FBE0F909D
:100C00001F901895E091C9009E2F9F5F903408F0C7
:100C100090E0F0E0E757FF4F80838091CA0098177B
:100C2000E1F39093C900559A08959091CA0020E08D
:100C30008091C900981709F421E0822F08951F922E
:100C40000F920FB60F9211242F938F939F93EF93D0
:100C5000FF93DF93CF930F92CDB7DEB78BB189832C
:100C600089818C7119F08EEF9FEF0EC0E0910B011E
:100C70009E2F9F5F903408F090E020910C01921716
:100C800041F457988AEA9AEA9093980180939701E1
:100C900013C0F0E08CB1E553FF4F808390930B01BC
:100CA000949B0AC0822F891B982F905C913408F482
:100CB000892F883008F494980F90CF91DF91FF919D
:100CC000EF919F918F912F910F900FBE0F901F90DA
:100CD000189590910B0120E080910C01891321E07F
:100CE000822F089590910C0180910B019817E1F3E8
:100CF000E92FF0E0E553FF4F2081E92FEF5FE0346B
:100D000008F0E0E0E0930C0194990BC080910B0196
:100D1000E81B8E2F805C813408F4E82FE83008F05F
:100D2000949A579A822F0895EE27FF27CF01EE2736
:100D3000FF273196D9F38099FCCFEE27FF27319614
:100D4000A9F30297809BFBCF0A97449678F7EE0FA2
:100D5000FF1FEE0FFF1F88279927019629F380991F
:100D6000FCCF882799270196F9F23197809BFBCF1A
:100D70003A977496E0F69C0183E0369527958A951C
:100D8000E1F72150304086E02238380718F42C3043
:100D9000310510F420E030E0C9010895949881B342
:100DA000826281BB88980E9494069C010097D9F3C7
:100DB000832F8F7780BD29B91BB888E98AB986E867
:100DC00080BD1092C9001092CA0010920B011092BF
:100DD0000C0101C08CB15F99FDCF949A08958823CE
:100DE00091F0C29AAF9B02C0AE9BA5988A988B984F
:100DF000979ABA9A8FEF8ABBAF9B02C0AE9B14C082
:100E0000AD9AA59A089592989398AF9901C0AE991A
:100E1000A5981ABABA9897988A9A8B9AAF9904C0EB
:100E2000AE9902C0AE9AA69A08958823A9F0AE9A08
:100E3000A99AA89A979902C0AE99A598A398AF9835
:100E4000969AA69AA19AA09A979902C0AE9902C0C2
:100E5000AD9AA59AC19A0895AB9AAE9A979B01C094
:100E6000AE9BA598A698A198A098AF9A9698A39A99
:100E7000979B04C0AE9B02C0AD9AA59AC1980895F5
:100E80001F920F920FB60F9211242F938F939F935F
:100E9000EF93FF9305B600FE35C090914E0120916F
:100EA0004D01921721F1E92FF0E0E35FFE4F8081C1
:100EB00080958BBB892F8F5F80934E01803410F01B
:100EC00010924E0180914F01882339F080914E019C
:100ED000821719F4AD9810924F0185B78E7F85BFA8
:100EE0008AB780648ABFC2988AE09AE006C08BB74E
:100EF0008F7B8BBFAD9A8FE09FE09093960180939C
:100F0000950103C08BB780688BBF7894FF91EF91F8
:100F10009F918F912F910F900FBE0F901F9018955A
:100F20001F920F920FB60F9211248F938BB78F776A
:100F30008BBF85B7816085BF8AB780648ABF8BB756
:100F400080648BBFC29A8F910F900FBE0F901F903D
:100F500018950BB606FC06C0F8948BB780648BBF5F
:100F60000E9440070895E0914D019E2F9F5F9034AD
:100F700008F090E0F0E0E35FFE4F808380914E0147
:100F80009817E1F390934D010E94A9070895E0910D
:100F90004D019E2F9F5F903408F090E0F0E0E35FFA
:100FA000FE4F808380914E019817E1F381E080939A
:100FB0004F0190934D010E94A90780914F01882312
:100FC000E1F70895809193011816C4F08BB78F7DD7
:100FD0008BBF81E00E94EF0610924D0110924E01EE
:100FE00010924F0185B7816085BF81E080939301A6
:100FF0008FE09FE0909396018093950108959091E2
:101000004E0120E080914D01981709F421E0822FD4
:1010100008951F920F920FB60F9211248F939F93F2
:10102000EF93FF9304B606FE15C084B78F7B84BF91
:101030008AB780628ABF9398909190019F5F9034A5
:1010400008F090E080919101981761F090939001E1
:10105000929A2DC092990AC08AEA90E090939801E2
:10106000809397018BB78F7D8BBF21C0929884B7F7
:10107000806484BF8AB780628ABF89B3E09190019F
:10108000F0E0E05BFE4F809580839D9909C08FEF73
:1010900090E0909396018093950181E08093920176
:1010A000939A8AEA90E09093960180939501FF913C
:1010B000EF919F918F910F900FBE0F901F901895F9
:1010C000409191012091950130919601809190017C
:1010D000522F632F2FEF30E04817C1F35093950143
:1010E00060939601E42FF0E0E05BFE4F9081E42FE7
:1010F000EF5FE03408F0E0E0E09391010BB605FC0F
:101100000EC0929908C0809190018F5F803408F0E2
:1011100080E0809390018BB780628BBF929A892F79
:1011200008958091930187FD25C090914D01809194
:101130004E018917E1F78BB78F738BBF80E00E9458
:10114000EF0610929001109291011092920184B7D3
:101150008F7B84BF8AB780628ABF8BB780628BBF68
:10116000929A8FEF809393018FEF90E09093960186
:101170008093950108959091900180919101891734
:1011800011F081E008958FEF90E0909396018093A5
:10119000950180E0089580919201882319F01092C2
:1011A000920181E008958BB78F718BBF80E00E9420
:1011B000EF0680E00E941507A89A10929301109202
:1011C000960110929501089581E00E94150780E034
:1011D0000E94EF061092930181E090E090939601B7
:1011E000809395010895282F80919301813031F4E7
:1011F00090914D0180914E018917E1F7222361F012
:10120000AF9B02C09799A598AE98AF9910C09799D7
:101210000EC0AD9AA59A0895AF9902C0979BA59864
:10122000AE9AAF9B04C0979B02C0AD9AA59A089551
:10123000882331F0A8988CE291E00197F1F70895A6
:10124000A89A0895A9988CE291E00197F1F7A99ADC
:10125000089580E00E94150780E00E94EF0610923A
:101260009301939AB99AA79A81B3806C81BB85B791
:101270008F6085BF8BB78F718BBF089580E690E03C
:101280009093AA018093A9019093AC018093AB0144
:101290008EE690E09093A8018093A70108951F9394
:1012A000FC01838185FD4FC00E94910880917C00E4
:1012B00090917D0097FF13C0809194018823E9F5F8
:1012C0000E946008182F0E94CB08882379F00E94A2
:1012D000BB08882359F481E08093940107C0182F3C
:1012E0008FEF9FEF90937D0080937C009091A10100
:1012F000992331F180919F01181711F58091940184
:101300008823D9F49230C8F00E946008182F809189
:10131000A0011817C1F00E94CB08882339F00E9461
:10132000BB08882319F481E08093940110937C001A
:1013300010927D0010919F0103C01092940103C090
:10134000212F30E002C02EEF3FEFC9011F91089519
:10135000CF93DF93EC010E94E2078FEFCF3FD807D6
:1013600081F58091A40120917E0030917F00882337
:10137000A1F037FD03C0822F0E94B3078091A40122
:10138000823038F08091A2010E94B3078091A301BE
:1013900002C08091A201282F02C037FD1EC08FEF2E
:1013A0009FEF90937F0080937E008091A601882319
:1013B00021F0822F0E94C70710C0822F0E94B3071E
:1013C0000CC080917E0090917F0097FD02C00E942A
:1013D000B307D0937F00C0937E00DF91CF91089533
:1013E00090E00E94A80980E090E008958FEF9FEFC1
:1013F0000E94A8090895FC01838185FD2AC080917F
:1014000080009091810097FF04C00E947206282FEF
:1014100007C0282F8FEF9FEF90938100809380006B
:1014200090919B01992399F080919901281779F463
:10143000923078F00E947206982F80919A01981746
:1014400041F090938000109281002091990130E04A
:1014500002C02EEF3FEFC90108952FEF8F3F920793
:1014600089F480919E01882379F080919C010E94EB
:10147000020680919E01823038F080919D010E9489
:10148000020608950E940206089590E00E942D0A27
:1014900080E090E008958FEF9FEF0E942D0A08955D
:1014A000803209F091118DC380528F55E0F7089575
:1014B000911187C3803219F089508550D0F7089573
:1014C0009111089581568A5108F4805285580895E3
:1014D000FC0183818F7C83830895CF93DF93EC019C
:1014E0004B8140FF1AC046FF0AC04F7B4B838E8161
:1014F0009F8101969F838E838A81282F2BC042FF74
:1015000013C0E881F9818081282F332727FD30958A
:101510002115310529F440624B832FEF3FEF1BC0AB
:101520003196F983E88311C0EA85FB85CE010995E0
:101530009C0197FF0AC09B812F5F3F4F11F080E213
:1015400001C080E1892B8B83E8CF8E819F8101963A
:101550009F838E8330E0C901DF91CF9108950F936F
:101560001F93CF93DF938C01EB018B8181FF1BC015
:1015700082FF0DC02E813F818C819D812817390704
:1015800064F4E881F9810193F983E88306C0E88572
:10159000F985802F0995892B31F48E819F810196E1
:1015A0009F838E8302C00FEF1FEFC801DF91CF91A1
:1015B0001F910F910895A0E0B0E0E1EEFAE00C94E5
:1015C000FF0DFE01359661917191A091A901B09135
:1015D000AA0113968C911397886013968C9380912F
:1015E000A9019091AA01AF010E949F0CE091A9016D
:1015F000F091AA012381277F23832096E2E00C94B7
:101600001B0E9C01FB01838180FF11C086FD0FC072
:101610009FEF2F3F390759F0228380648F7D8383AA
:101620008681978101979783868330E002C02FEFF0
:101630003FEFC9010895FC0120FD08C023FD05C04E
:1016400022FF02C073836283518340830895EF9227
:10165000FF920F931F9344FF02C033E011C046FF77
:1016600002C034E00DC0DB01FC01AA0FBB1FEE1F5E
:10167000FF1F1094D1F76A0F7B1F8E1F9F1F31E051
:10168000660F771F881F991F3150D1F77B018C019E
:10169000E20EF11C011D111DA8019701B701CA013D
:1016A0001F910F91FF90EF9008950F931F93CF9389
:1016B000DF938C01C8010E946D0AEC0197FD08C000
:1016C0000E94580A892BB1F7CE01B8010E94010B84
:1016D000CE01DF91CF911F910F910895A0E0B0E06E
:1016E000E4E7FBE00C94F70DEC01C62E5A01122F33
:1016F0000E946D0AAC018B3219F08D3251F41068E2
:10170000CA9409F46DC0CE010E946D0AAC0197FD28
:1017100067C06DEFD62ED1228D2D807301F5403339
:10172000F1F4CA9409F447C0CE010E946D0AAC01DD
:1017300097FD41C082E0D82A483711F0483559F466
:1017400080E4D82ACA94B9F1CE010E946D0AAC0196
:1017500099232CF430C0D6FC02C080E1D82AEE24B4
:10176000FF248701242F2053283088F0D4FC09C09F
:101770002A3068F0D6FE05C02F7D822F8151863039
:1017800028F0CA01BE010E94010B12C02750C801F7
:10179000B7014D2D0E94270B7B018C0182E0D82AD6
:1017A000CA9461F0CE010E946D0AAC0197FFDACFB6
:1017B000D1FC04C015C0EE24FF248701D7FE08C069
:1017C00010950095F094E094E11CF11C011D111D91
:1017D000C501B801A7012D2D0E941B0B81E001C09E
:1017E00080E0CDB7DEB7EAE00C94130EA0E2B0E0E3
:1017F000ECEFFBE00C94F30D6C01A62E8A0179014D
:10180000FE01319680E2DF011D928A95E9F770E0D2
:1018100030E060E040E050E04F01A1E0B0E0F601D0
:101820008381F70183FD259183FF21917F0122238D
:1018300009F47EC02E3519F44115510569F1872F41
:1018400090E08417950744F42D3551F12D3221F4A1
:10185000332329F431E021C0332309F4622F322FDE
:10186000832F869586958695F401E80FF11D832FC9
:1018700087703D0102C0660C771C8A95E2F72081D3
:1018800026292083361711F430E007C0361710F4EC
:101890003F5FE6CF3150E4CF71E04F5F5F4FBFCF86
:1018A000332319F08E8180628E83772359F0FE01F5
:1018B00031969E012F5D3F4F808180958193E21785
:1018C000F307D1F7BB24B3944E010894811C911CFB
:1018D000C6010E946D0AAC0197FD22C086958695CF
:1018E0008695F401E80FF11D808190E09A01277040
:1018F000307002C0959587952A95E2F780FD05C066
:10190000CA01B6010E94010B0BC00115110519F0A7
:10191000D8014D938D01AA94BB24AA20C9F602C018
:10192000BB2031F40115110529F0F801108202C025
:10193000EE24FF24C701A096EEE00C940F0EA0E069
:10194000B0E0E5EAFCE00C94F30D5C016B013A01B8
:10195000FC01178216828824EAC0812F90E00E9441
:10196000580A892B21F0C5010E94550BE0C01532A1
:1019700049F4F601F3FC6591F3FE61916F01653264
:1019800069F415E2C5010E946D0A97FDDCC01817C5
:1019900009F4CDC0B5010E94010BDAC06A3219F01A
:1019A000162F00E006C0F3FC1591F3FE11916F01B4
:1019B00001E099240FC00260692D70E080E090E0A2
:1019C00040E20E94270B962EF601F3FC1591F3FEE0
:1019D00011916F01212F20532A3068F301FD03C0BC
:1019E00099249A9403C0992009F4B2C0183621F0C2
:1019F0001C3699F4F6010BC0F601F3FC6591F3FE79
:101A00006191683619F06F01162F07C008600460F5
:101A1000F3FC1591F3FE11916F01112309F498C0A5
:101A200085EC91E0612F70E00E94E40D892B09F4B0
:101A30008FC0802F00FF03C0EE24FF2407C0F301F6
:101A4000E080F18022E030E0620E731E1E3651F419
:101A5000F5014681578160E070E0C701202F0E94A8
:101A60001B0B65C0133691F481FD02C09924939439
:101A7000C5010E946D0A97FD66C0E114F10419F0DA
:101A8000F70181937F019A9499F74FC01B3559F460
:101A9000C501692DA70196010E94F60B6C01009704
:101AA00009F043C03DC0C5010E94550B97FD4BC0D6
:101AB0001F3659F1103728F4143629F1193639F543
:101AC00027C0133719F0153711F51DC0C5010E9445
:101AD0006D0AEC0197FD11C00E94580A892B29F06C
:101AE000CE01B5010E94010B08C0E114F10419F008
:101AF000F701C1937F019A9449F7E114F104A9F029
:101B0000F701108212C0006203C0006101C00064CE
:101B1000C501692DA701202F0E946E0B882329F48F
:101B2000F5018381807379F413C000FF8394F5017C
:101B3000F380F601F3FC1591F3FE11916F0111236F
:101B400009F00BCF05C0882019F42FEF3FEF02C03A
:101B5000282D30E0C901CDB7DEB7EEE00C940F0EB2
:101B6000DC01CB01FC01E199FECF06C0FFBBEEBB5F
:101B7000E09A31960DB20D9241505040B8F7089559
:101B8000DC01A40FB51F4150504048F0CB01840F39
:101B9000951F2E910E94D10D41505040D0F70895CD
:101BA000262FE199FECF9FBB8EBBE09A01970DB225
:101BB000021631F02DBB0FB6F894E29AE19A0FBEEF
:101BC0000895992788270895FC010590061621F0AD
:101BD0000020D9F7C00108953197CF0108952F92C1
:101BE0003F924F925F926F927F928F929F92AF92AD
:101BF000BF92CF92DF92EF92FF920F931F93CF93FA
:101C0000DF93CDB7DEB7CA1BDB0B0FB6F894DEBF90
:101C10000FBECDBF09942A88398848885F846E84B6
:101C20007D848C849B84AA84B984C884DF80EE8000
:101C3000FD800C811B81AA81B981CE0FD11D0FB609
:101C4000F894DEBF0FBECDBFED010895F894FFCF2D
:101C50000000000300000000450AFB09000000002E
:101C6000000300000000F0094F090000FFFFFFFF24
:021C7000FFFF74
:02000004008278
:020000003FC1FE
:02000004008377
:01000000EB14
:00000001FF
